:030000000219FDE5
:03000B000200A848
:03002B0002015D72
:03005B000202DCC2
:030073000202C2C4
:1000800002030406080C10182030406080040608A3
:100090000C10182030406080A0C000070F1F3F05E3
:1000A000050D050205030302C2AFC0D0C0E0206207
:1000B00017E5256002E473E525F4F58A758B00D217
:1000C00062D0E0D0D0D2AF3285268AC262E526F473
:1000D000602F758B00D0E0D0D0C297C295C293D26A
:1000E000AF32C297C295C293206E0C206609740E7F
:1000F000D5E0FDE57E4290758B00D0E0D0D0D2AF48
:1001000032758A00C28DD26201F701B730680520CE
:100110006602D29701B7306805206602D29501B712
:10012000306805206602D29301B7C29630680A2073
:100130006607740CD5E0FDD29701B7C29430680A07
:10014000206607740CD5E0FDD29501B7C2923068E5
:100150000A206607740CD5E0FDD29301B7C2AFC286
:10016000AD53E6EFC0D0C0E0D2D3D2AFC2CEE52AC5
:100170006007207449152A21BE7800790020742E6A
:10018000E580307E01F430E30278FF53DACF207E41
:100190000343DA20307E0343DA10C2D8C271E5800F
:1001A000307E01F430E30279FFC3E89970CB30610F
:1001B00003752A18207403752A18885FD27020747A
:1001C0000DE52B6004152B21CE43DA01C2D8207037
:1001D000024130A85F206102C270207431C3E894EC
:1001E000F0400374F0F8E8C4540F28F87984B7039A
:1001F00002410EC313C3138721200802C313200A30
:1002000006C3C898F8410E28F8500374FFF8C3E8F5
:1002100095685003E568F88822E52D54066011E5DD
:1002200033C313C31324062522F52250037522FF7E
:10023000852224A824C3E52495644002A864882567
:10024000E56970024174C3E8AA699A5003E8FAE4C8
:10025000F9EAC333FBE56BF45B29400D256AF8E549
:100260006A6002156A400B41740AC3E56A9A50023B
:10027000056A78FF8826C3E52594404002D26420B1
:10028000CF0AD0E0D0D043E610D2AD32C2CF053A8B
:100290007801E52A6005307402152AC3E55F9401F0
:1002A000400575620041B8756300756C00E5622415
:1002B00001F56250037562FFD0E0D0D043E610D262
:1002C000AD32C2AFC0D053E67FC260759100855693
:1002D00094855795759104D0D0D2AF32C2AF53E612
:1002E000EFC2ADC0D0C0E0C0F0D2D3D2AFA8FBA95E
:1002F000FCC2D8307102614353DACF207E0343DA67
:1003000010307E0343DA20D271E580307E01F42084
:10031000E302611A88278928A16A53DACF207E0375
:1003200043DA20307E0343DA10C2D8C2713074023F
:10033000A1567800E580307E01F430E302A15688B2
:100340005FA13E53DACF207E0343DA20307E0343A1
:10035000DA10C271206102811C53DACF207E034380
:10036000DA10307E0343DA20C2D8D271885A895B12
:10037000C3E89558F8E99559F97B007E087A00C3DF
:10038000E8948CE994005005755E00810E88217810
:10039000A2E6A8216055C3E894C8E994005008E497
:1003A000D2E4FB7A0A61E9C3E89468E99401500851
:1003B000E4D2E3FB7A0F61E9C3E894D0E9940250F8
:1003C00008E4D2E2FB7A1E61E9C3E894A0E994054F
:1003D0005008E4D2E1FB7A3C61E9C3E89498E994DF
:1003E000085008E4D2E0FB7A787E00C3E8955CFC14
:1003F000E9955DFD30E70AECF42401FCEDF43400EE
:10040000FD755E00C3EC9AED9E5003755E01885C3D
:10041000895D855A58855B597802A13EC3E89527C6
:10042000F8E99528F9307C02A122307B02A1223024
:100430007A02A11B207502813FE9FDE8FC815EE99B
:10044000C313F9E813F8307902A11BE9C313F9E8E3
:1004500013F8307802A11BE9C313FDE813FC2061F7
:1004600026C3EC941CED940240028175ED7018C314
:0E047000EC94C850120529C3E529940A5002E5
:10047E00A156755F00D270A156E529600215297844
:10048E0088E6F97400207F087896B90302789EE614
:10049E0024FAFEE43400FFC3EC9EFCED9FFD9208AF
:1004AE00B90310A2085007207609D27681C13076A2
:1004BE0002C276A2085016B9030DECF42401FCED2D
:1004CE00F43400FD0204DB78007900A122B9031593
:1004DE00EC33FCED33FDC3EC940AFCED9400FD50BF
:1004EE00047C007D00C3EC94FFED9400400678FF81
:1004FE007900A122EC8575F0A4C5F0A2F733F87946
:10050E0000400302053E78FF790002053EE9C31361
:10051E00F9E813F8307C0EE9600278FFC3E813386F
:10052E00F8E43400F9C3E894FFE99400400278FF40
:10053E00885FD270206102A156741FF4552F4BF5BF
:10054E002FC274EB7002D274752A18307403752A98
:10055E000A306102A16A20740353DAFE2074037517
:10056E002B06D0F0D0E0D0D0D2AD43E610327901D8
:10057E0002059A790302059A790A02059A791E02F2
:10058E00059A796402059A79C802059A7817E4D516
:10059E00E0FDD8FAD9F6227A147B780205C17A10DA
:1005AE007B8C0205C17A0D7BB40205C17A0B7BC828
:1005BE000205C17902B27DE4C294D5E0FDD295D593
:1005CE00E0FDC295D5E0FDD294D5E0FDD297E5765B
:1005DE00D5E0FDC2977496D5E0FDD9D9EAF8D5E0FD
:1005EE00FDD8FBDBCEC29422C37C007D0075F000EB
:1005FE0005F0EA33FAEB33FB50F6EB13FBEA13FA92
:10060E00C3E9FFE8FEE89AF8E99BF95004EFF9EE2A
:10061E00F8B3EC33FCED33FDD5F0DFEDF9ECF82259
:10062E00E889F08A20D2D4F8A9F07B0030F70B7B52
:10063E00FFF42401F8E9F43400F9E88520F0A4ADC4
:10064E00F0F8E98520F0A4AFF0FEED2EF974003F2E
:10065E00FA7C04C3EA13FAE913F9E813F8DCF48B15
:10066E00F030F70AE8F42401F8E9F43400F9E889E7
:10067E00F0C2D4F8A9F02222C3E54113F9E54013E4
:10068E00F8C3E54598F8E54699F9500CC3E894800F
:10069E00E994FF40160206BDC3E8947FE99400502A
:1006AE00030206BD787F79000206BD788079FF8847
:1006BE004A894B22E54A2547F8E54B3548F9854BE3
:1006CE0020E4300701F43549FA30E709C3EA94F023
:1006DE0040150206FBC3EA940F50030206FB78FF97
:1006EE0079FF7A0F0206FB780079007AF0C3E524D1
:1006FE009564500AC374019524500B020719E54BFB
:10070E0020E70E020719E54B30E706884789488A2D
:10071E00492278A4E6FAC3E54A33F8E54B33F9D11A
:10072E002EE930E70BC3E89480E994FF4013E153C0
:10073E00C3E8947FE994005002E153787F7900E199
:10074E0053788079FFE820E715C3E52398F8400930
:10075E00C3E89401400302077A780102077AE8F4AD
:10076E0024012523F8400302077A78FF884C22786B
:10077E00A5E6FAA848A949D12EE930E70CC3E894BA
:10078E0001E994FF40160207AEC3E894FFE9940016
:10079E0050030207AE78FF79000207AE780179FFA9
:1007AE00E920E715C3E54C98F84009C3E8940140E9
:1007BE00030207D578010207D5E8F42401254CF889
:1007CE0040030207D578FF88242278FFC26420698F
:1007DE003D206A12D264C3E541940A4009C3E5255F
:1007EE0094405002C26479A1E76023E541601F7412
:1007FE00FF8541F0848539F0306A0375F005A4F861
:10080E00C5F0600278FFC3E895675002A867886656
:10081E0022C3E5409440E5419401E566500314017E
:10082E0030046002F566220208382275E8902278BC
:10083E0083E6FFE5E820ECF7A8BDA9BE0573C3E586
:10084E007394084052757300E9FA79A0E76044EAA0
:10085E007007E574601B020873C3E895746010E5B9
:0F086E00745006600C1402087F0460F902087FC2
:10087D00E574F574C394A8401B7564C0C39405401A
:10088D0013756480C39405400B756440C394054093
:10089D000375640075BB0122E564F460020564E52F
:1008AD0073B4070375BB1E22743279A687F0A4C5F5
:1008BD00F0A2F733F8C3E895644002A86488228853
:1008CD0024882588268867227540007541F022C24C
:1008DD00AF75C820A8CCA9CDAA3A30CF010A75C8EA
:1008ED0024D2AFAB3BAC3C883B893CC3E89BF8E9D9
:1008FD009C206908F930670221F1214EAD3D8A3DFA
:10090D00F9EA9DFA600478FF79FFAE3EAF3F8B3E6A
:10091D008C3FC3EC9FFCC3E99CF542A83BA93CC3AB
:10092D00E89EF8E99FF9C3E54113FBE54013FAE8AA
:10093D002AF540E93BF54150067540FF7541FF2111
:10094D0098AA40AB41AC40AD417E047F02C3EB940D
:10095D000440021E1FC3EB940840021E1FC3ED137B
:10096D00FDEC13FCDEF7C3EA9CFAEB9DFBEF60098F
:10097D00C3E913F9E813F8DFF7EA28FAEB39FB8A34
:10098D00408B4150067BFF8B408B41C3EB94025053
:10099D0002D2673069047F0321C37892E6FFC3E575
:1009AD0037948240110FC3E53794A040010FC3EF78
:1009BD00940640027F057E06E541C4540FF9E541DA
:1009CD00C454F0F8E540C4540F28F8C3E89EFAE982
:1009DD009400FB4009C3EA9402EB940050047A02A0
:1009ED00E4FB413DAA40AB41EBC4FEEAC4540F4EBB
:1009FD00FCC3EA9CFAEB9400FBC3E813C313F8EABB
:100A0D0028FAEB3400FB8A408B41C3EB9402400281
:100A1D00C2677806EBC4FE7B00EAC4540F4EFAC3DE
:100A2D00EA98FA4005C3940250027A027892E6FFE2
:100A3D00306002413D855256855357D26043E68062
:100A4D00C3E49AF8E49BF930670241D7E8FAE9FB71
:100A5D00D3E913FDE813FC88528953C3EF94036067
:100A6D0038EF20E00DE82CF8E93DF9ECFAEDFB024A
:100A7D000A92E828F8E939F9C3E82402F8E93400C4
:100A8D00F97AFE7BFFC3EF9403400E8A548B558891
:100A9D004E894F8C508D51610B885489558A4E8BE0
:100AAD004F8C508D51306920C3E53394034019E5C7
:100ABD0042A2E713F8E555F4240138400B20E7086E
:100ACD007554FFF42401F555610BE8FAD3E813FCD6
:100ADD008852C3EF94036020EF20E007E82CF8EC78
:100AED00FA41F7E8282402F87AFEC3EF9403400890
:100AFD008A54884E8C50610B88548A4E8C50E56B0D
:100B0D00C3335002646BF56B3060026115753402AE
:100B1D00D26043E680E52D54066026A840A941C366
:100B2D00E913F9E813F8C2AF53E67F759100C3E4FA
:100B3D0098F594E499F595759104D26043E680D2C9
:100B4D00AF22D265754400752000306B03752040CF
:100B5D00020B6ED265754400752040306B03752015
:100B6D0000D2AF7801206722E52D54066002C265E0
:100B7D00C3E5419405401378029405400878039429
:100B8D000540027806306902780A206019E5446054
:100B9D001530690AC3E53394034003D53406D2AF4B
:100BAD00D26C8148711DD2AF0000C2AF206726E51F
:100BBD0041C3FB940F40027B0FEB240530730123DF
:100BCD00306A02742820620123F93069027982E5C6
:100BDD008BC39940B50544E59E7005E59B020BEF6F
:100BED00E59A5440B52002813230690A08C3E89471
:100BFD000A4001086197206502616EC26553E67F68
:100C0D007591003067107594007595FE759104D23D
:100C1D006043E680616EAE40AF41C3E49EF594E45F
:100C2D009FF5958119C3E53394025002616E3065CD
:100C3D0002616ED80281466197C26C53E67F759151
:100C4D0000855494855595759104854E56854F575D
:100C5D00D26043E680D2AFE52D54066008206A02CB
:0E0C6D000533020C82306C0D206B0A206507E7
:100C7B001581158102152422780030640530650238
:100C8B007801E53775F007A4F9E5F028F5F0E9A24E
:100C9B00F013A2F113A2F213F537C3947850037536
:100CAB003778C3E53795384008D266C297C295C2EC
:100CBB009330600281BC855056855157D26043E614
:100CCB008022207D14C2AF754302C294D296D2AF5C
:100CDB00759F33759E00020EAEC2AF754302C29470
:100CEB00D292D2AF759F33759E00020EAE30724317
:100CFB00207D20C2AF75430390013B757E10C293DC
:100D0B00C292306204D295A116D294D2AF759E22B4
:100D1B00020EAEC2AF75430390013B757E10C297B6
:100D2B00C296306204D295A136D294D2AF759E236F
:100D3B00020EAE207D17C2AF754303900116C2930E
:100D4B00306202D295D2AF759E22020EAEC2AF7543
:100D5B004303900116C297306202D295D2AF759EB3
:100D6B0023020EAE207D11C2AF754304C296D29200
:100D7B00D2AF759E23020EAEC2AF754304C292D2A0
:100D8B0096D2AF759E22020EAE307249207D23C2E1
:100D9B00AF75430590012A757E40C295C2943062AF
:100DAB0004D297A1B2D296D2AF759F33759E000233
:100DBB000EAEC2AF75430590014C757E04C295C251
:100DCB0094306204D293A1D5D292D2AF759F337572
:100DDB009E00020EAE207D1AC2AF75430590010C2A
:100DEB00C295306202D297D2AF759F33759E0002C7
:100DFB000EAEC2AF754305900120C2953062E8D2AA
:100E0B0093D2AF759F33759E00020EAE207D11C23B
:100E1B00AF754306C292D294D2AF759E22020EAE2C
:100E2B00C2AF754306C296D294D2AF759E23020E03
:100E3B00AE307242207D20C2AF75430190014C75DC
:100E4B007E04C297C296306204D293C15AD292D218
:100E5B00AF759E23020EAEC2AF75430190012A758A
:100E6B007E40C293C292306204D297C17AD296D29C
:100E7B00AF759E22C1AE207D16C2AF7543019001A6
:100E8B0020C297306202D293D2AF759E23C1AEC2FD
:100E9B00AF75430190010CC293306202D297D2AF6F
:100EAB00759E22C2662290010A757E00C297C2957A
:100EBB00C293C296C294C292C26222788076FF0815
:100ECB0076FF0876FF0876FF087603087604087627
:100EDB0008087601087601087601788C7601087689
:100EEB00FF0876FF0876FF0876FF0876FF08760383
:100EFB000876FF0876FF0876FF0876250876D00877
:100F0B0076FA0876FA0876040876FF0876010876F2
:100F1B000008767A0876FF087601087601087600D5
:100F2B00087603227887E6FFC2727888E6C39403BB
:100F3B006008C27DE630E102D27DC27E7889E63060
:100F4B00E102D27EC3EF94026008758E01D2730268
:100F5B000F62758E00C273227880E6149000809326
:100F6B0078A4F67881E6149000809378A5F67886BD
:100F7B00E61490008D9378A6F6789CE67538FF758D
:100F8B00390CB402067538A075390AB403067538E6
:100F9B008275390578A3E61490009A93F569D1B15F
:100FAB0022227896E6FA7897E6FB7888E6B4030572
:100FBB00C3EB940EFB307F047A007BFFC3EB9AFCF0
:100FCB00C3948250027C827575000575EC8575F0B3
:100FDB00A4C3E5F0947D40F222D27FF1AD12058BD4
:100FEB007A007B007C10120581E55F2AFA74003BC6
:100FFB00FBDCF37C04C3EB13FBEA13FADCF7FEC256
:10100B007F120FAD22E5EF20E6037520000520903F
:10101B003DFFE520146006901FFF146000930460F1
:10102B000375EF1253D9BF7581C043FF8012057C46
:10103B0075EF0243B203E5B3240420E70DF521E578
:10104B00B120E0068521B343B101120EB1758008C2
:10105B0075A40075F1FF75D4F775900275A5FC7535
:0E106B00F2FD75D50075A0FF75A60075F300A7
:1010790075D60075B0FF75A70175F4FF75E241E4F7
:10108900F8F6D8FD756B01120EC6121566789886AA
:1010990076753001C2AF1205951205A512058B129E
:1010A90005AC12058B1205B312058B12167F1205BA
:1010B90095120595120590C2AF78FA79FA3083072F
:1010C900D9FBD8F7021C00120F2F120F63120FACB5
:1010D900120FAD78988676120EB1758850758912FF
:1010E90075C82475910475D84075A82275B802751C
:1010F900E690759B80759D00759A80759C0075D1E9
:101109000E75BC5875BB0175BA1F75E88012057C50
:10111900D2AF12083553DACF207E0343DA20307E6E
:101129000343DA1043DA01C2D8C271120595D261BC
:101139007B037A0CE55E70077A0CDB030210C012A0
:10114900058B2070030210C0C270E55FC394024092
:10115900E1E52F541F856160F561B560D5DAD5C227
:101169006153DACF207E0343DA20307E0343DA105D
:10117900C2D8C27178A2E67008D274E52F54E0F59E
:101189002FC275752900120590307409C3E5299499
:101199000A4002D27512058178023074027800C3C0
:1011A900E55F9840F0C2AF1205A51205A51205A585
:1011B900D2AF120595754D007888E6B4030241A6B1
:1011C900120581788CE6C3940150030212A6E5301A
:1011D900C3940150030212A6207435C3E55F94FF3E
:1011E90050030212A6C2AF1205BAD2AF120590C3BC
:1011F900E55F940150EFC2AF1205A51205861205ED
:10120900A5D2AF120590C3E55F94FF40E902170428
:101219007F05D27F120FAD120590C2AFC27F120FA8
:10122900ADAE5FC3E55F947FD2AF407B12057CC250
:10123900AF1205BAD2AFDFDA120FE4C3EE94057824
:1012490097F61205951215A81216877F0AD27F12F2
:101259000FAD120590C2AFC27F120FADAE5FC3E5ED
:101269005F947FD2AF50E412057CC2AF1205A5127C
:1012790005861205A5D2AFDFD4120FE4EE24057856
:1012890096F61205951215A81216B6120590120FA8
:10129900ADC3E55F94FF500221E1021704C3E55F86
:1012A900954D4003855F4D12059078017988E7B423
:1012B90003027805C3E55F98400221C1C2AF120558
:1012C900BA1205BA1205BAD2AF120595753000E403
:1012D900F531F5320531E531F470390532789AE6A0
:1012E9007819146012783214600D787D14600878CA
:1012F900FA146003753200C3E53298401715327548
:1013090031B478998676C2AF1205BAD2AF78988689
:1013190076120590120586E52A700530740201C01F
:1013290078012074027806C3E55F9840A77888E6BB
:10133900C394036003120590E52A70030210C0C22A
:10134900AF120EB1E4F522F523F524F525F526F5BE
:101359006AD2AF7885E6C333F568E4F545F546F515
:1013690047F548F549F573F52CF52DF537757308EB
:1013790075BB1E12057C120839E5E820ECFBA8BDF7
:10138900A9BEE97001F8887412083D75730875BB28
:101399001E7887E6FE7602120F2F7887EEF6C2AF27
:1013A9007564FF1208B5852264852265852266D297
:1013B900AF75220175240175250175260185636CB8
:1013C900756D017888E6B40307C27D307602D27D57
:1013D900D268D269753300120E17120E3C1208D565
:1013E9001208DC1208D51208DC1208D5021405C24D
:1013F900AF120F2FD2AF75730075BB01120B6012BC
:101409000685120C83120CCD1208DC120B4F306DBD
:10141900031206862067031207D830670312081FD4
:10142900120C83120CF81208DC120B60306D0312D7
:1014390006C2120C83120D6F1208DC120B4F306DAD
:1014490003120720120C83120D941208DC120B6090
:10145900306D0312077D120C83120E171208DC126D
:0E1469000839120B4F120C83120E3C12083D74
:101477001208DC306932206B2F85676485676585C4
:10148700636C756D0179187A0CC3E53399400CC20A
:1014970069D26A8A357564FF0214AFC3E55F9401A8
:1014A700400302140502152C306A1B206B18E53522
:1014B700147004C26A61F8F535C3E55F940140030F
:1014C70002140502152C753600C3E5627882985020
:1014D70054307404E52A604D7888E6B40317207DFC
:1014E7000520760781FC30760281FC206B07D26BE2
:1014F700856764814478F0306B058567647820C31D
:10150700E5419850028105306B1BC26BC27D307676
:1015170002D27DD26A75351285676481050536E585
:101527005F6002A12F753600C2AF120EB17887E651
:10153700FE7602120F2F7887EEF6E4F522F523F5F3
:1015470024F525F526F568C268D2AF12057C120E80
:10155700B1307409C3E5369405400201C041D89003
:101567001A0D78201215EAE520B45A0CA31215EAD1
:10157700E520B4A503021588120EC61215A8021598
:10158700A7901A0378807B0A1215EAA308DBF99063
:101597001A0F788C7B181215EAA308DBF9901A2723
:1015A70022C2AF121629121603901A00740E1215D2
:1015B700EFA374041215EFA374141215EF901A0316
:1015C70078807B0A1215EEA308DBF9901A0F788C46
:1015D7007B181215EEA308DBF912163C12161A90A7
:1015E7001A2722E493F622E6438F01538FFD75EF06
:1015F7000275B7A575B7F1F0538FFE22438F0243EB
:101607008F0175EF0275B7A575B7F1901A0DF053F5
:101617008FFC22901A0D745AB1EF901A0E74A5B16F
:10162700EF227A3079D07820901A40B1EAE520F796
:1016370009A3DAF7227A3079D0901A40E7B1EF0997
:10164700A3DAF922AB77A878BB01027984BB02023F
:101657007985BB03027986BB04027992BB050279BF
:1016670087BB060279A3BB0702799CBB080279886E
:10167700BB09027989E8F7227C05120595DCFB2274
:10168700C2AF1205A51205AC1205B31205BA1205B1
:10169700861205A51205AC1205B31205BA12058606
:1016A7001205A51205AC1205B31205BAD2AF22C2B4
:1016B700AF1205BA1205B31205AC1205A5120586BD
:1016C7001205BA1205B31205AC1205A5120586124A
:1016D70005BA1205B31205AC1205A5D2AF22AE7733
:1016E700AF78C2AF1205A51205A51205A51205868A
:1016F700DEF21205BA120586DFF8D2AF22D187D102
:101707007FD17F757701757801757900D1E57C0503
:10171700AD5F120595C3ED955F70F5C3E55F940165
:10172700400AC3E55F94FF4032021740D14BB1A88E
:10173700D187C2AF75EF12D17FDCD50579C3E579C3
:101747009403500280C6D17F0578E5771490009FF7
:1017570093F808C3E57898500280AED17FD17F0512
:1017670077C3E577940A5002809C120EC6B1A8C2CF
:06177700AF75EF12D17FF7
:0319FD00021010C5
:101A00000E0414FFFFFFFF0304080101015AA501A2
:101A1000FFFFFFFFFF03FFFFFF25D0FAFA04FF01DE
:081A2000007AFF01010003FF41
:101A4000235467794B4637304148562320202020C5
:101A500023424C48454C4923463331302320202033
:101A60002020202020202020202020202020202076
:101C0000C2AFC2D353D9BF7581C043B20343FF8073
:101C1000752438752503B1C975EF0275E24043F1AB
:101C20000853A4F775D400D2837DFA780379E67C53
:101C300010752200752300901DD67B0675249875BB
:101C400025013083028142208308D8FBD9F9DCF7D3
:101C500081B4308308D8FBD9F9DCF781B4B189E4C9
:101C600093A3C39A6004DDC381B4DBDBB17B600264
:101C7000812B7B08E493FAA3B15CDBF87A30B15C8A
:101C8000752200752300B17BEAFCEBFDC3ED94FEE9
:101C9000400EB17B8A278B28ED30E0048A828B834B
:101CA000B17B7AC270D8C3ED94FE601350CEBD00F4
:101CB00025EC60097520007521FF0200008100A855
:101CC00027A9280809D804D90281D3B17FEA89AAB3
:101CD000F281C50D81A0C3ED94035049EDA2E092BD
:101CE000007AC5C3E5829400E583941C50902000DF
:101CF00010438F02438F0175B7A575B7F1F030001F
:101D00001FA827A9280809438F01538FFDD804D99C
:101D100002A12089AAE275B7A575B7F1F0A3A10DBC
:101D2000538FFC817C7AC1BD030CE493A3FAB140CC
:101D3000DCF8B138817C817EAA22AB23B15CEBFA5E
:101D4000EA6222752608C3E52313F523E52213F57D
:101D50002250066323A0632201D526EAB1C9B1C986
:101D600075260AEAF4200102D283300102C283B14F
:101D7000C9C3134002C201D526EB22B17FEAFB2082
:101D80008302A17F308302A184752608AE24AF258B
:101D9000C3EF13FFEE13FEB1CDB1C9C3EA13308315
:101DA000024480FA30E703632201C3E52313F523DD
:101DB000E52213F52250066323A0632201D526D91C
:101DC000E52265236523F52222AE24AF250E0FDE22
:101DD000FEDFFCD20122424C48656C693437316326
:041DE000F3100601F5
:00000001FF
